:1000000007309F00B32288237C2B82075034493469
:10001000433453344D3454345734583420347634C4
:1000200032342E3431340034501C2928A1234C1C86
:100030001628C6001B3A03191F2846081628B6239F
:10004000C6001B3A03191F284608773A0319BA2B32
:1000500016281030BF00C101C0012030BB00A22013
:1000600044080310C1070318C00ABF0B2F28A701BB
:100070004008A6004108A500BA207D30AF0020301E
:10008000AE00AD01AC0191218830AF00AA30AE00C6
:10009000AD01AC01FC2136212708C6002608C700A7
:1000A0002508C800A71F5928A709A609A5092D30AA
:1000B000BB002608A7002508A6000330B5003E3087
:1000C00086224608A7004708A6004808A500BA20CF
:1000D0007C30AF003830AE005130AD00EC30AC00B9
:1000E00091218430AF00AE01AD01AC01FC2136217D
:1000F000C601A71F7F28A709A609A5094614250838
:10010000A6000330B500383086222D304618B600E0
:1001100008301723093017233608C0223708C022B9
:100120003808C0220A3017233B08C0223C08C022EE
:100130003D08C0222E30C0223E08C0224330C022DB
:10014000CE22212B2030C3003630C200C501C401AD
:10015000031100008618C50A0319C40AC30BA92895
:10016000C20BAA280310C50DC40DC50DC40DC50DC5
:10017000C40D08009630A800A901A71FC828A5092A
:10018000A609A709A50A0319A60A0319A70AA91708
:10019000B3012708031DDD282608A7002508A600AF
:1001A000A501B3152708031DDD282608A700A60111
:1001B000B311331627080319EE283308A802031DCC
:1001C000031CEF290310A71BEB28A50DA60DA70DF7
:1001D000A80BE328EF29A91FA7130034A701A60144
:1001E000A501A401A8010034B3012708031D1429A7
:1001F0002608A7002508A6002408A500A401B31519
:100200002708031D14292608A7002508A600A50114
:10021000B31133162708031D14292608A700A601C9
:10022000B31527080319EE283308A802031D031C81
:10023000EF290310A71B2329A40DA50DA60DA70DBB
:10024000A80B1A29EF292A1B251CEB28A41FEB2831
:10025000A50A0319A60A0319A70A031DEB28A70C70
:10026000A60CA50CA80A0319E429EB2828080319F1
:1002700000342708A900A7179630A802A81F8529CF
:10028000A809A80A08302802031C6129A800A50DA6
:100290002608A5002708A600A70108302802031C8D
:1002A0006129A800A50D2608A500A601083028028E
:1002B000031C6129A800A50DA5012808031D031032
:1002C0006A29280803196A290310A70CA60CA50C93
:1002D000A80B64292A1B251C7629031C7629A50A4C
:1002E0000319A60A0319A70AA71B8529A91F003409
:1002F000A709A609A509A50A0319A60A0319A70AA9
:100300000034A701A601A50100342A14AA1FFF3456
:10031000A701A91FFF30A700A600A500A90DA70CE3
:10032000FF342808031D2F080319EE2827082E067E
:10033000A9002F08A8077E30031CA229A8020318D1
:10034000E429A529A802031CEF292708A4002608F0
:10035000A3002508A200A417AE170310A701A60149
:10036000A5011830B300221CBF292C08A5072D08B1
:1003700003182D0FA6072E0803182E0FA707A70C8A
:10038000A60CA50CA40CA30CA20C0310B30BB32950
:10039000A71BCF29A40DA50DA60DA70DA8032A1BE9
:1003A000251CE129A41FE129A50A0319A60A03199E
:1003B000A70A031DE129A70CA60CA50CA80A03197E
:1003C000E429A91FA7130034AA14AA1FFF34FF3081
:1003D000A800A700A600A500A90DA70CFF342A15A8
:1003E000AA1FFF340130A800A701A601A501A90D8D
:1003F000A70CFF348030AE0627082E06B300A401F8
:10040000AB0128082F02031C1D2A2F08A200280870
:10041000AF002208A8002E08A2002708AE0022087C
:10042000A7002D08A2002608AD002208A6002C086F
:10043000A2002508AC002208A5002F0803190034EB
:100440002708A900A717AE172F082802AF00031925
:10045000502A08302F02031C462AAF002C08AB009C
:100460002D08AC002E08AD00AE0108302F02031C91
:10047000462AAF002C08AB002D08AC00AD010830B7
:100480002F02031C462A2908A70000342F0803194D
:10049000502A0310AE0CAD0CAC0CAB0CAF0B492AC0
:1004A000B31F5D2AAB09AC09AD09AE09AB0A03194C
:1004B000AC0A0319AD0A0319AE0A2B08A4072C08CD
:1004C00003182C0FA5072D0803182D0FA6072E08BB
:1004D00003182E0FA707B31B762A031C2329A70C8A
:1004E000A60CA50CA40CA80F2329E4290318F428B2
:1004F000A409A509A609A709A40A0319A50A0319AD
:10050000A60A0319A70A8030A906C8288400AE01EC
:100510000A30AD0093222208800030308007840327
:10052000B50B872A0800A301A2011030B400270DE3
:10053000A20DA30D2D08A2022E08031C2E0FA3024C
:100540000318A92A2D08A2072E0803182E0FA307A7
:100550000310A60DA70DB40B972A0034CA000000A3
:10056000CA0BB02A08008316061383120613003044
:100570000023C900F022CF0007300023D00008007C
:10058000CC000A30CB0003100613031C06174908E1
:10059000AE220314CC0CCB0BC42A08000D30C02AA9
:1005A00008000A30C02A08002030C02A08004C1079
:1005B000861E00340930CB004F08AE220310861E81
:1005C0000314CC0C4908AE220000CB0BDE2A4C08E9
:1005D000861AE82A4C140800D7224C1CEC2A080082
:1005E000CD00CE010310CD0C4D080319FE2ACE0715
:1005F000CD0C4D080319FE2ACE02F22A4E0808003F
:100600007F3983169B001C141A08831208007F3957
:1006100083169B008B131C1555309D00AA309D003E
:100620009C141C118B179C18132B83120800002399
:10063000C60046080023003803190800C022C60A75
:10064000192B06191428D7224C1C212BC6001B3A43
:1006500003192C2B4608212BEC22C6001B3A031948
:100660002C2B4608443A03195F2B46084F3A0319CE
:10067000522B4608563A03197C2B4608503A031968
:10068000582B4608553A03196E2B46084D3A031964
:1006900014284608723A0319D22B4608513A031916
:1006A0000028212B1430C70008300023C600612B1E
:1006B0001430C700C02208300023C600722BC601C8
:1006C000C701EC2283169A00831246080723C7034A
:1006D0000319212BC60AC61F612B212B8030C02293
:1006E000C601C70146080023C022C7030319212BF6
:1006F000C60AC61F722B212BC601460805200038EA
:100700000319852BC022C60A7D2BCE22D122212B94
:1007100083168617A7308100831205130230002349
:10072000F10001300023F00003300023D100043039
:100730000023D20005300023D30006300023D4006C
:1007400008004C10861F00340930CB004F08AE2241
:100750000310861F0314CC0C4908AE220000CB0BFB
:10076000A82B4C08861BB22B4C140800A1234C1C50
:10077000B62B080083162130A000200884008312C5
:10078000B6238316841780008413A00A201FCC2B65
:10079000A01ECC2B201ACF2B7106031DBD2B83125C
:1007A0000830172383162130A000D50120088400CB
:1007B0008417000884138312C60052084606031DDE
:1007C000E62B0B3017230430D500ED2BD503031D8A
:1007D000EB2B2E30C0224608C0228316A00A201F11
:1007E000F52BA01EF52B201AFB2B84170008841371
:0C07F0007106031DD62B8312CE22212B94
:02400E00223D51
:1042000052002100430074000D00620068000000AD
:104210000C0021002E003D00210035003000300050
:1042200033002E00300030004E002F0030003100EF
:104230003400320037002E003000300045005F00AF
:1042400000003000300030002F003000300030001F
:10425000670030003000300074000000580050004B
:1042600049004300200053004D005400200074001A
:1042700065006D0070003A000000580050004900D1
:1042800043002000570058002000740065006D00B6
:0642900070003A0000007E
:00000001FF
